:020000040802F0
:1040000000C00020AD5E0208296002087D61020840
:104010008D610208916102089561020800000000AC
:104020000000000000000000000000000000000090
:104030000000000000000000000000000000000080
:104040000000000000000000000000000000000070
:104050000000000000000000000000000000000060
:104060000000000000000000000000000000000050
:104070000000000000000000000000000000000040
:10408000000000000000000000000000996102082C
:104090009D61020800000000000000000000000018
:1040A0000000000000000000000000000000000010
:1040B00000000000A16102080000000000000000F4
:1040C00000000000000000000000000000000000F0
:1040D00000000000000000000000000000000000E0
:1040E00000000000000000000000000000000000D0
:1040F00000000000000000000000000000000000C0
:1041000000000000000000000000000000000000AF
:10411000000000000000000000000000000000009F
:10412000000000000000000000000000000000008F
:1041300010B505F0ADF802F075F94FF07E5104F0BE
:10414000F1FF0B4905F0F8F80A4904F0EDFF0A49C0
:10415000044605F0ADFA38B92046064905F08AFA5A
:1041600000B1044C204610BD034C204610BD00BFDA
:10417000D1C69B4200000C420000B94308B5FFF7CE
:10418000D7FF4FF07C5104F0CFFF05F09BFA08BD3C
:104190002DE9F047002082B09F4CE0F73BF850201B
:1041A000DD214FF6FF720023009400F04DFEDFF892
:1041B0009C82DFF89C92DFF89CA205270A2505EB7C
:1041C00085067600AE420BDD2C462046FFF7D6FF73
:1041D00064192821DC22102301F02AF8A642F4DC1D
:1041E0002846FFF7CBFF2621DC221F2301F020F811
:1041F000B5F57A7F11DA2846FFF7C0FF0C38182191
:10420000002380B24FF6FF72CDF800A0019500F0B8
:104210001BFE013F16D03546D1E72846FFF7AEFF1B
:1042200089FB0523E9170C38C1EBA31580B21821CF
:1042300000234FF6FF72CDF80080019500F004FED8
:10424000013FE8D1754E764F6FF0400435E02046CF
:1042500005F01EF8734904F067FF734905F06CF828
:10426000724904F061FF7249054605F021FA002801
:1042700040F0B98028466D4905F0FCF9002800F0AF
:10428000BB8023204FF4B97128221F2300F094FF34
:10429000664D4FF07C51284604F046FF05F012FAB7
:1042A000C11F0020019489B246F2EC720346053426
:1042B000009700F0C9FD0A2C32D086FB043CE517BC
:1042C000C5EBAC0202EB8200B4EB400FBFD020463E
:1042D00004F0DEFF534904F027FF534905F02CF8A2
:1042E000524904F021FF5249054605F0E1F9002842
:1042F00077D128464D4905F0BDF900B14B4D4FF03F
:104300007C51284604F010FF05F0DCF90534024624
:10431000102323204FF4B97100F04EFF0A2CCCD1AA
:104320000024444D4E21234646F2FF726FF0590699
:104330004FF4BB700095019600F086FD7B2123466B
:1043400046F2FF724FF4BB700095019400F07CFDC3
:1043500000955A250195384DA821234646F2FF7253
:104360004FF4BB7000F070FDD5212346009546F256
:10437000EC722046314D00F067FDD521234646F210
:10438000FF724FF4BB70009500F05EFD23462C4C8D
:1043900018214FF6FF724FF4B970009400F054FDED
:1043A00023494FF6FF740B462648274A009400F035
:1043B000FBFD1E4923480B46234A009400F0F4FD00
:1043C00020481B490246194B009400F0EDFD1E48A1
:1043D00017490246154B009400F0E6FD02B0BDE817
:1043E000F087134D8BE723204FF4B971DC221F2394
:1043F00000F0E2FE0E4D4CE74FF07C51284604F0F1
:1044000093FE05F05FF94FF4B97102461F23232094
:1044100000F0D2FE3DE700BFBC9702086766666603
:10442000E897020800008C42000010400000204283
:1044300000005C43EC970208F0970208F49702082A
:10444000F897020800000C420000B943E097020808
:10445000D34D6210DC9702082DE9F04F304E83B047
:1044600000F036FF2F4800F0A5FF3368002B51DD28
:104470002D4FDFF8CCA0341D00254FF47A781FE0D3
:10448000D4F808B00135584605F01CF92749814693
:10449000584604F051FF05F015F90028B8BF404216
:1044A0008AFB0031C317C3EB611C642202FB1C02B0
:1044B00049461F4800F07EFF30680C34A84229DDD1
:1044C0006168D4F800900846019105F0FBF819499D
:1044D0008346019804F030FF05F0F4F80028B8BFD7
:1044E000404287FB0032C317C3EBA21108FB110344
:1044F0005A464946104800F05DFFA06801F016FFDB
:104500000028BDD10D4800F055FF306801350C344E
:10451000A842D5DC03B0BDE8F04F00F025BF00BFD6
:1045200004310020FC970208D34D62100000C842FD
:104530002898020800007A44189802083098020867
:104540001F85EB512DE9F04F91B0FFF721FE24209C
:104550000121DFF77BFE05200021DFF777FE092030
:104560000121DFF773FE04210A20DFF76FFE4FF40D
:104570007A7001F075F90A210D910020974C0146DF
:10458000024603460094964D00F05EFC00204FF674
:10459000FF7201460346934E009500F055FC002340
:1045A00033600D9804F074FE01464FF07E5004F025
:1045B00077FF002701468C480B9701F0AFFF0B9F58
:1045C0000C90DFF82482B9467BE00798874905F014
:1045D00051F808B1854A079285490F9804F0A4FD67
:1045E0004FF07C5104F0A8FE804904F09DFD814904
:1045F000064605F05DF8002840F0A98030467B496A
:1046000005F038F800B1794E4846002105F028F849
:10461000002800F0A48073490B68B3F5C87F0EDA58
:1046200003EB4302DDF83C906E4801EB820C5F1C0B
:10463000CCF80440CCF80850CCF80C9007606E4BD6
:104640006E4958460093019404F076FE05F03AF85E
:104650000290284605F036F869490390284604F090
:104660006BFE05F02FF8674A0028B8BF404282FB76
:104670000047C1176423C1EB671403FB14050F98AF
:10468000049505F01FF80590002001464FF6FF72D3
:10469000034600F0D9FB0420DFF7DCFD4FF6487B32
:1046A000584540F0C1800C99404604F045FE5649FB
:1046B000804604F0E9FF002800F0CB80079F0B96AE
:1046C000D146404604F0FEFF01F028FB04460A20D4
:1046D00001F0C6F80FA9204601F072FA4B49834653
:1046E00004F0DEFE01F09EFE494904F025FE054679
:1046F000204604F0CDFD474904F01EFE464904F073
:104700001BFE0F9904F010FD394906460F9004F086
:10471000CFFF20B13046404904F004FD0F90204601
:10472000FFF706FD3D498246284604F0FDFC3C4962
:1047300004F002FE2D4904F0F7FC2E49079004F026
:10474000B7FF00283FF441AF2A48079044E74846A6
:104750000021284E04F084FF00287FF45CAF394626
:104760005246079B484646F2EC77009700F01CFC47
:1047700031460B9804F0D6FC0021074604F098FF60
:10478000E0B1012338461E49099304F073FF099BE9
:10479000E8B1D9B200293FF43EAF0F9801F0C6FD51
:1047A00000283FF438AF46F2FF7E48460B99524648
:1047B0003346CDF800E000F0F7FB2CE70122384645
:1047C0001849099204F074FF099B0028E1D10023E5
:1047D000D9B200293FF41FAFDFE700BF34980208C9
:1047E0007C98020804310020000020410000204293
:1047F0000000344300005C43A498020800007A449F
:104800000000C8421F85EB51005043487B146E3FA7
:104810000000A041BD3706350000B44300008C42C3
:10482000000010400000C8C20020454D014602466D
:1048300003460095434E00F007FB002001464FF66B
:10484000FF720346009600F0FFFA4FF4FA6001F0A1
:1048500007F800243C4E3D4F009601973C4D3D4EDD
:104860003D4F204621464FF6FF723C4B0295039682
:104870000497059400F00AFB002856D0012859D06F
:1048800002283FF47AAE03282BD00428E2D1344822
:1048900000F0ACFD2A4E054621462246234620461E
:1048A000304F009600F0D0FA204621464FF6FF72B6
:1048B00023460097019500F0C7FA2846FFF7CCFD84
:1048C000002829D0284F204621464FF6FF72234664
:1048D0000097019500F0B8FA4FF47A7000F0C0FF2D
:1048E000B8E7224800F082FD154E054621462246D3
:1048F000234620461B4F009600F0A6FA204621468C
:104900004FF6FF7223460097019500F09DFA284666
:1049100000F090FE0028D5D1154D21464FF6FF72CC
:104920002346009500F090FAD6E7FFF731FC0A2005
:104930000D9022E63224FFF72BFC0D941DE600BFFC
:1049400034980208D0980208E4980208EC9802080B
:10495000F4980208009902080C990208DC980208F1
:1049600060990208289902083899020818990208E3
:1049700048990208CB7970B49842CE682AD30122B4
:1049800003FB02F2B0FBF2F49C42F9D2E2B1002543
:1049900002FB1400B2FBF3F20DB9002C0FDD092C61
:1049A00016DD0B7A002B0CBF572337231C1906F892
:1049B000014B4AB1CB790135B0FBF2F4E8E7002AAC
:1049C000FAD1303406F8014B0020307070BC7047CB
:1049D0003023EBE701220446D9E700BF2DE9F84375
:1049E000D36817461A7805460E463C68A2B1002CDB
:1049F00012DD13F8010F013C04F0010160B15CB15C
:104A000009B104E044B113F8011F013C21B113F8CE
:104A1000012F013C002AF5D1797901B1013CBB7924
:104A20002BB1FB79102B61D0082B08BF013C3879E2
:104A300010BB631E002C6CDD20214FF001082846BE
:104A400003EA0809B047A04513D0B9F1000F06D01A
:104A5000202128464FF00208B047A04509D0202168
:104A60002846B04708F1020820212846B047A04553
:104A7000F5D179794FF0FF34002934D1B97921B1DA
:104A8000FB79102B34D0082B3FD03A7902B3002C9D
:104A90001EDD30214FF00108284604F1FF39B047F0
:104AA000A04509EA080913D0B9F1000F06D030215A
:104AB00028464FF00208B047A04509D030212846CB
:104AC000B04708F1020830212846B047A045F5D18B
:104AD000FC68217829B12846B04714F8011F002945
:104AE000F9D1BDE8F8832846B047C7E7023C9EE706
:104AF00028463021B04797F808C02846BCF1000F7F
:104B00000CBF78215821B047BFE728463021B04775
:104B1000BBE71C46B0E700BF43688268013393429D
:104B200005D20268436002F8011B026070474360CF
:104B3000704700BF2DE9F04188B0984605AB0646A6
:104B40000D461446049300272178002942D00134F1
:104B500025293AD101978DF8097038463B4614F85B
:104B6000011B002936D0232963D030295FD0A1F161
:104B700030025FFA82FCBCF1090F8DF808008DF855
:104B80000A3012D80023D0B2A1F1610C09285FFAD3
:104B90008CFC22D9A1F14102BCF1050FD2B225D87B
:104BA000A1F157020A2A18DD01936C2908BF14F8F5
:104BB000011B69294BD03ED8632969D044D85829B4
:104BC0001DD0C1D831B12529BED13046A8472178A2
:104BD0000029BCD108B0BDE8F08114F8011B03EB3B
:104BE000830002EB4003A1F13002CCE7052ADBD8B9
:104BF000A1F13702D6E775293BD07829A4D1A1F1DC
:104C00005801D1F1000C4CEB010E10208DF80B0077
:104C10008DF80CE0D8F8000001A9FFF7ABFE304694
:104C2000294601AA08F10408FFF7D8FE8CE7012005
:104C300095E7012393E773291FD0DCD86F2983D12F
:104C400008238DF80B30E5E764297FF47DAF0A2354
:104C50008DF80B30D8F8000008F1040800281EDB9E
:104C600001A9FFF787FE3046294601AAFFF7B6FEE5
:104C70006AE70A218DF80B10CCE7D8F800303046EF
:104C8000294601AA08F104080493FFF7A7FE5BE791
:104C900098F80010304608F10408A84754E72D2280
:104CA000404201A98DF80920FFF764FE30462946ED
:104CB00001AAFFF793FE47E710B584B001900024E6
:104CC000039101A804490294FFF734FF019B1C7073
:104CD000029804B010BD00BF194B02080CB410B507
:104CE00082B004AC54F8042B23460194FFF7E4FF90
:104CF00002B0BDE8104002B0704700BF70B4027847
:104D0000002A47D0254C0023E51D202107E090F81C
:104D100000C004F803C010F8012F01331AB32E2A83
:104D2000F5D10130072BF2DC5E1EA219D343EE1839
:104D3000531CAB42517006F001060AD01EB103F8B5
:104D4000011FAB4205D05A1C59700233AB4251705F
:104D5000F9D190F800C0082304F803C010F8012F1F
:104D60000133002ADBD10A2B11DC5A1C20210A2A2C
:104D7000E15403F001030ADC1BB1A15401320A2AF9
:104D800005DC501CA15402320A2A2154F9DD0348E3
:104D900070BC70471346014CE7E700BFC8430020D2
:104DA0009CF802302DE9F0416446154613B10246E5
:104DB00008461146C1F30F21C0F30F20DFF726FA92
:104DC000DFF752FAC5F580721E49550081FB0537A1
:104DD0002388C7EBE57C03F4FC640CF58075E610D2
:104DE00006FB05F6DA0003F4784700F4FC613F1295
:104DF00002F0FF04C5F5807CCA1004FB05F407FB34
:104E000005F50CFB026200F47843C10018120CFB9C
:104E10000050002A01F0FF01B8BFFF320CFB014136
:104E200093125A010028B8BFFF30C312002942EA8A
:104E3000C320B8BFFF3140EAE12188B2BDE8F041AC
:104E4000DFF7E6B9565555552DE9F04385B00DF11C
:104E5000300E5EF804CB0C4C06460F4615469846BD
:104E60006246734637212046CDF80CE0FFF724FF59
:104E7000394681462A46304643460094DFF7E4F936
:104E8000484605B0BDE8F083D443002008B42DE9BE
:104E9000F04F88B011AF57F8045B00F11003029790
:104EA000039002983E4F041D119588469246059343
:104EB0004FF0000904944FF6487B0020394D4146DD
:104EC000024603460095FFF7BFFF119C414652463C
:104ED000002303980094DFF7B7F9119804F03EFC23
:104EE000029A049914680791002C57D0059E00255A
:104EF00006EBC006C9EB050EDEF1000C4CEB0E0311
:104F0000B0B2414652460094DFF79EF9204604F0C5
:104F100025FC079902300C680B1D06EBC006013515
:104F20000793002CE6D164223A803B889CB2002C87
:104F3000FBD10420DFF78EF980F47E4C8CF4A4744E
:104F400048F2480104EA01000028F2D00420DFF70B
:104F500081F95845FAD164223A80B7F800E01FFA87
:104F60008EF3002BF9D114F0080F05D0B9F1000F22
:104F700002DD09F1FF39A0E714F4004F05D0013D2F
:104F8000A94502DA09F1010997E714F0400F94D01E
:104F9000484608B0BDE8F04F01B070472546C2E76B
:104FA0005C850020349802082DE9F04F83B0144648
:104FB000BDF8302088461E464FF087410023ADF8EB
:104FC00004208DF8063004F0B7F904F07BFB4FF0B5
:104FD00087410746204604F0AFF904F073FB4FF019
:104FE00087410446404604F0A7F904F06BFB4FF0FC
:104FF00087418146304604F09FF904F063FBE31BD0
:10500000C9EB000283EAE375A5EBE37582EAE2717E
:10501000A1EBE2718D4280F2CB80BA46012798461F
:10502000A3468DF80670134604464F46BC4205DA87
:10503000D1463846DA462746CB46044607F1800C6F
:105040002CF0FF054FEA0828EA1B98FBF3F808FB51
:1050500002F10029B8BFFF310AEB212A0CF0FF0052
:105060000AF0FF07C7F5807EC0F5807606FB0EF3D9
:1050700006FB07F62AF0FF091A12284649460DF1E9
:10508000040CFFF78DFE3212284609F580710DF1F0
:10509000040CFFF785FE04F1800222F0FF09C4EB47
:1050A000090708FB07F4002CB8BFFF340BEB242CD6
:1050B0000CF0FF0702F0FF06C7F5807106FB01F355
:1050C00006FB07F62CF0FF041A120DF1040C4846FB
:1050D0002146FFF765FE0135320A0DF1040C484602
:1050E00004F58071FFF75CFE4D455EDA0AEB0806B9
:1050F00026F0FF0706F0FF0AEC4328463946CAF5BA
:1051000080720DF1040CFFF74BFE04EB090B2846EF
:1051100005F580740DF1040C07F580715246FFF718
:105120003FFE4C45CBF3002B06EB08053DDABBF107
:10513000000F0AD025F0FF0705F0FF06204639468C
:10514000C6F580720DF1040C20E025F0FF0705F094
:10515000FF0620463946C6F5807245440DF1040C21
:10516000FFF71EFE204607F5807132460DF1040C54
:1051700004F5807425F0FF0705F0FF06FFF710FE29
:105180003946C6F580720DF1040C2046FFF708FE83
:1051900020460DF1040C07F58071324604F5807449
:1051A000FFF7FEFD4C454544CFDB03B0BDE8F08F73
:1051B00090468346CA4639E788422DE9F0410546C4
:1051C0000C461E462DDC97B23946C0EB040880B26F
:1051D000DFF71CF802353046DFF71AF8AC42C8F3A7
:1051E000400820DBB8F1000F09D0A8B23946DFF73C
:1051F0000DF802353046DFF70BF8AC4215DB3946C7
:10520000A8B2DFF703F802353046DFF701F8A8B29D
:105210003946DEF7FBFF02353046DEF7F9FFAC42D8
:10522000EDDABDE8F081BDE8F081BDE8F08100BFB6
:1052300091422DE9F0410C4615461E462DDC87B201
:1052400089B23846C4EB0208DEF7E0FF023430468C
:10525000DEF7DEFFA542C8F3400820DBB8F1000FFF
:1052600009D0A1B23846DEF7D1FF02343046DEF76E
:10527000CFFFA54215DBA1B23846DEF7C7FF0234E7
:105280003046DEF7C5FFA1B23846DEF7BFFF023475
:105290003046DEF7BDFFA542EDDABDE8F081BDE89E
:1052A000F081BDE8F08100BF08B5FFF727FD074B8F
:1052B000014603F5277203F1440003F52973DEF775
:1052C000E5FFD0F1010038BF002008BDC843002031
:1052D00010B5FFF713FD0C4C014604F5297304F1DA
:1052E000440004F52772DEF7CFFF0023C11A4842BD
:1052F00040EB010084F8A802C4F8AC32C4F8B03224
:10530000C4F8B43210BD00BFC843002038B5144CF7
:1053100094F8A8327BB1D4F8B032D4F8AC22E118BA
:1053200001330132B3F5007F81F84400C4F8B03294
:10533000C4F8AC2200D238BDD4F8B4020025421C17
:1053400004F5277104F14400C4F8B052C4F8B42243
:10535000DEF7A0FF0028EED084F8A85238BD00BFC9
:10536000C84300200846D1E738B5104C94F8A8028D
:1053700018B919E02020FFF7C9FFD4F8B032002B8C
:10538000F8D10B48D4F8B4120025490200F5167282
:1053900000F5187384F8A852DEF77EFFC5EB000C09
:1053A000DCF1000040EB0C0038BD00BFC84300201A
:1053B0000C4400200FB470B582B006AE56F8042B32
:1053C000084C002008493346D4F8AC520196FFF748
:1053D000B1FBD4F8AC02401B02B0BDE8704004B091
:1053E000704700BFC84300206553020870B50646E9
:1053F000002409E00D48FFF771FC0C48FFF754FF4B
:1054000090B1B4F57A7F0FD023460D21324607487C
:10541000FFF764FC0548FFF747FF651C0D210234C8
:1054200032462B460028E5D1004870BD804600205A
:105430002DE9F00FC20000F4FC64E41002F0FF025A
:1054400000F478410912A4F1FC05A2F1F80685EAFE
:10545000E579A9EBE57986EAE678A8EBE678A1F1AB
:10546000F80C8CEAEC77A7EBEC77A01809EB0803B3
:105470004018DB19984200F3DA8003460020A4F1BB
:10548000800BA2F18008A1F1800788EAE879A9EBF6
:10549000E8798BEAEB7AAAEBEB7ACA4487EAE779F8
:1054A000A9EBE779D1444B45C4BF4B46022086EABD
:1054B000E67AAAEBE67A04EB0A0909EB010A5345FE
:1054C000C4BF5346032085EAE579A9EBE57909EBEA
:1054D000020A0AEB01094B45C8BF4B4604EB020A1E
:1054E000C8BF04208CEAEC79A9EBEC79D1444B4598
:1054F000C4BF4B46052086EAE679A9EBE67985EA42
:10550000E57AAAEBE57ACA440AEB01094B45C4BF28
:105510004B46062085EAE57AAAEBE57A92448CEAC6
:10552000EC79A9EBEC79D1444B45C4BF4B4607203D
:1055300086EAE679A9EBE679BCF1000FB8BFCCF1B9
:10554000000CA144E1444B45C4BF4B46082088EA07
:10555000E87CACEBE87C04EB0C0909EB010C63453F
:10556000C4BF634609208BEAEB79A9EBEB7909EB21
:10557000020C0CEB01094B45C4BF4B460A2004EB5F
:10558000020987EAE77CACEBE77CCC446345C4BF07
:1055900063460B2085EAE57CACEBE57CB8F1000FB7
:1055A000B8BFC8F10008E04487EAE77CACEBE77CD1
:1055B000C4446345C4BF63460C20002EB8BF764286
:1055C000002DB8BF6D42AD19002FB8BF7F42EF1953
:1055D000BB42C8BF3B46A2F1600CC8BF0D20BC3C1B
:1055E00084EAE476A6EBE476BCF1000FB8BFCCF118
:1055F000000C6039664481EAE175A5EBE175751927
:10560000AB42C4BF2B460E20B83A002CB8BF644250
:10561000002AB8BF5242A4180029B8BF494204EB7F
:10562000010C9C45B8BF0F20BDE8F00F704701206A
:1056300025E700BF2DE9F041FFF74AFE874C04F152
:1056400036066078651CFFF761FE02346878FFF764
:105650005DFEB442F5D10020FFF758FE0020FFF7B1
:1056600055FE0020FFF752FE0020FFF74FFEF82006
:10567000FFF74CFEFC20FFF749FEF820FFF746FE3F
:105680000020FFF743FE8020FFF740FE8020FFF759
:105690003DFE8020FFF73AFE0020FFF737FE002096
:1056A000FFF734FE0020FFF731FEF820FFF72EFE53
:1056B0000020FFF72BFE0020FFF728FEFC20FFF75D
:1056C00025FE0020FFF722FE0020FFF71FFEF82036
:1056D000FFF71CFE0020FFF719FE0020FFF716FE63
:1056E0000020FFF713FE0020FFF710FEFC20FFF75D
:1056F0000DFEF820FFF70AFE0020FFF707FEF82056
:10570000FFF704FEFC20FFF701FE0020FFF7FEFD7F
:105710000020FFF7FBFDF820FFF7F8FD0020FFF762
:10572000F5FDF820FFF7F2FD0020FFF7EFFD002068
:10573000FFF7ECFD0020FFF7E9FD8020FFF7E6FD15
:105740000020FFF7E3FD0020FFF7E0FD8020FFF7DA
:10575000DDFD0020FFF7DAFD0020FFF7D7FD8020F8
:10576000FFF7D4FD0020FFF7D1FD0020FFF7CEFDAD
:105770000020FFF7CBFD8020FFF7C8FDFC20FFF7DE
:10578000C5FD8020FFF7C2FD0020FFF7BFFD802090
:10579000FFF7BCFDFC20FFF7B9FDF820FFF7B6FDD1
:1057A0000020FFF7B3FD6020FFF7B0FDBC20FFF73E
:1057B000ADFD6020FFF7AAFD0020FFF7A7FD6020E8
:1057C000FFF7A4FDBC20FFF7A1FDB820FFF79EFD69
:1057D0000020FFF79BFD4FF0000840F291171FFAE1
:1057E00088F50124601E294680B2DEF70FFDDEF742
:1057F0003BFDFFF71DFE294606462046DEF706FD67
:10580000DEF732FDFFF714FE40EA0613D8B2FFF7C9
:105810007DFDA11C8CB2621E90B22946DEF7F6FC1B
:10582000DEF722FDFFF704FE294606462046DEF796
:10583000EDFCDEF719FDFFF7FBFD023440EA061030
:10584000C0B2A4B2FFF762FDBC42CBD108F101089F
:10585000B8F1F00FC3D1BDE8F04185E56F990208BA
:10586000034B1880188882B2002AFBD1704700BF12
:105870005C850020000000002DE9F04F40F66A78BA
:10588000044608FB00F00028B8BF033087B07A4E0A
:1058900004928210B6FBF2F6784D0293731C95FBCE
:1058A000F3F5059140F66A7795FBF4F197FBF1F07B
:1058B00005FB00F2202092FBF4F301460193DEF792
:1058C000C5FC07200021DEF7C1FC08203146DEF7C9
:1058D000BDFC00208021DEF7B9FC694A516801292E
:1058E000FCD1674A5768012FFCD006200121DEF762
:1058F000ADFC0320DEF7AEFC0028FAD0002602360D
:10590000DEF798FCDEF796FC962EF8D1204603F0E1
:10591000BFFC5C4903F010FD8146284603F0B8FC4B
:105920000146484603F0BCFD019C0390002C40F367
:10593000988000260024B146A046FF272EE003F001
:10594000A7FC0546204603F0A3FC039903F0F4FCF2
:10595000824600F0B1FC8346504600F025FD002150
:10596000824603F0E9FC0146584603F0DBFB0146A2
:10597000284603F0E1FC0146484603F0D5FB0AF156
:1059800000418146284603F0D7FC0146304603F02B
:10599000CBFB019A01349442064614D0DEF74AFC50
:1059A000029D5FFA80FC6046E045B8BFE04667456F
:1059B000A8BF6746002DC2D1049B002BBFD1019A1E
:1059C00001349442EAD1019B059C03EBD370C7EBF1
:1059D00008072760401003F05BFC0546294648464F
:1059E00003F05EFD29460446304603F059FD21468A
:1059F0000546204603F0A0FC29460646284603F04B
:105A00009BFC0146304603F08FFB00F039FF049900
:105A1000064621B11C4903F043FD049A1060029927
:105A200041B130464FF0804103F042FE28B9174B98
:105A30000298036007B0BDE8F08F05F100412046F1
:105A400000F0EEFC124903F077FC03F029F808A3FC
:105A5000D3E9002303F0A2F903F010FB029B1860C6
:105A6000E8E700264FF00008B146FF27ABE700BF8C
:105A7000182D4454FB210940FFA14A0400A24A0406
:105A800044040240DB0FC940F304B53F0000C07F6F
:105A90000000344310B5002182B004460A20DEF72E
:105AA000D5FB0220FFF7DCFE00221346204601A9A9
:105AB000FFF7E2FE019BC72B73DD01210A20DEF711
:105AC000C5FB0220FFF7CCFE0022204601A91346A9
:105AD000FFF7D2FE0198C72865DD02210A20DEF714
:105AE000B5FB0220FFF7BCFE002201A920461346A9
:105AF000FFF7C2FE0199C72957DD03210A20DEF70F
:105B0000A5FB0220FFF7ACFE00221346204601A9A8
:105B1000FFF7B2FE019AC72A49DD04210A20DEF709
:105B200095FB0220FFF79CFE00221346204601A9A8
:105B3000FFF7A2FE019BC72B3BDD05210A20DEF704
:105B400085FB0220FFF78CFE0022204601A91346A8
:105B5000FFF792FE0198C7282DDD06210A20DEF707
:105B600075FB0220FFF77CFE002201A920461346A8
:105B7000FFF782FE0199C7291FDD07210A20DEF702
:105B800065FB0220FFF76CFE00222046134601A9A8
:105B9000FFF772FE019AC72ACCBF0820072002B087
:105BA00010BD0020FBE70120F9E70220F7E7032002
:105BB000F5E70420F3E70520F1E70620EFE700BF53
:105BC00070B50C4682B0234601A96A460646FFF727
:105BD00053FE019B143BD22B13D8104D0720DEF748
:105BE00039FB2A6802EB820100EB8100006903F0B7
:105BF0004FFB009903F0A0FB094903F051FC02B0F0
:105C000070BD3046FFF746FF044D01A928606A4683
:105C100030462346FFF730FEE0E700BF00300020AB
:105C200000247449AFF300802DE9F041044610468A
:105C3000884603F02DFB374903F07EFB05464046BE
:105C400003F026FB0146284603F02AFCB8F1000FBA
:105C500007465CDD0020002618F0010F05463AD10A
:105C60002D4903F069FB2C4903F05EFA03F050FD67
:105C7000394624F8020B284603F056FA2549054612
:105C800003F016FD20B12846224903F04BFA0546E1
:105C9000284600F089FB01261DE000F085FB1E4927
:105CA00003F04AFB1C4903F03FFA03F031FD39468B
:105CB00024F8020B284603F037FA1649054603F08C
:105CC000F7FC144918B1284603F02CFA054628467B
:105CD00000F06AFB0136104903F02EFB0E4903F079
:105CE00023FA03F015FD394624F8020B284603F089
:105CF0001BFA0849054603F0DBFC0136054918B1DB
:105D0000284603F00FFA054646452846C5D1BDE8AA
:105D1000F08100BFDB0FC94000E0FF444FF4FA5CA4
:105D20002DE9F0410CFB00F42249651EA1FB05168C
:105D3000B20C0132204BB4FBF2F7B3FBF7F74FF68E
:105D4000FF784745A8BF47461C4D791C95FBF1F6E7
:105D500002FB06F606EB5004DFF86C80184BB4FB30
:105D6000F0F44FF0000EB4F5FA5FA8BF4FF4FA5408
:105D7000144DA3F828E040462146FFF755FF2B6855
:105D80000F2023F001022A602146DEF75FFA0E2081
:105D90004146DEF75BFA29680D2041F001032B60D4
:105DA0003946DEF753FA06EB5400B0FBF4F0BDE8D9
:105DB000F08100BF83DE1B43FFA14A0400A24A0416
:105DC00000140040440402409046002010B50D4CE1
:105DD0000021B4FBF0F4621C12F0010F08BF14465E
:105DE0001020DEF733FA1120611EDEF72FFA1220A1
:105DF0006108DEF72BFA044963085818B0FBF4F089
:105E000010BD00BFFFA14A0400A24A042248234952
:105E100070B4884223D0224CA14220D2024652F8CC
:105E2000046B0B46CD4343F8046B6519A342C5F3DD
:105E3000800514D23DB1156800F108021D6001F122
:105E40000803A3420BD2104650F8045B194641F8F0
:105E5000045B5568021D5D600B1DA342F3D3114A1C
:105E60001148824216D200211346D44343F8041B42
:105E700004198342C4F380040CD224B1196002F1E6
:105E80000803834206D21A4642F8041B5960131DC8
:105E90008342F8D370BC7047809E02080030002017
:105EA000043100200431002078850020054B064A8B
:105EB000DFF818D09A60FFF7A9FFDEF7D7F9FEF7F1
:105EC00041FBFEE700ED00E00040020800C00020BA
:105ED000F0B50A2883B009D00E4C27683F2F07D0B1
:105EE000E11901370871276003B0F0BD094C27683C
:105EF000094D0026E7193E71084F334629880A20CC
:105F00004FF6FF720097DEF79FF92B6826600E3B75
:105F10002B60E9E710850020043000201485002064
:105F200010B50446007828B1FFF7D2FF14F8010F2E
:105F30000028F9D110BD00BF10B50446C078000993
:105F4000092839DD3730FFF7C3FFE17801F00F0092
:105F5000092839DD3730FFF7BBFFA278100909287F
:105F600039DD3730FFF7B4FFA37803F00F000928BD
:105F700039DD3730FFF7ACFF60780009092839DDDB
:105F80003730FFF7A5FF94F801C00CF00F00092887
:105F900039DD3730FFF79CFF21780809092839DC03
:105FA0003030FFF795FF227802F00F00092839DC26
:105FB0003030BDE810408BE73030FFF789FFE178E3
:105FC00001F00F000928C5DC3030FFF781FFA2780F
:105FD00010090928C5DC3030FFF77AFFA37803F0F9
:105FE0000F000928C5DC3030FFF772FF6078000928
:105FF0000928C5DC3030FFF76BFF94F801C00CF0C6
:106000000F000928C5DC3030FFF762FF217808094E
:106010000928C5DD3730FFF75BFF227802F00F005B
:106020000928C5DD3730C4E7704700BF002038B508
:106030000146DEF7EBF83F484BF68031DEF7F4F827
:106040003C484BF68031DEF7EFF800210320DEF705
:10605000FDF8394C3948FFF763FF3948FFF760FF17
:1060600004F14400FFF768FF3648FFF759FF606C02
:1060700000251830FFF760FF3348FFF751FF606CD1
:106080001430FFF759FF3148FFF74AFF606CFFF704
:1060900053FF2F48FFF744FF606C0430FFF74CFFBD
:1060A0002C48FFF73DFF606C0830FFF745FF2A489A
:1060B000FFF736FF606C0C30FFF73EFF2748FFF715
:1060C0002FFF606C1030FFF737FF2548FFF728FFE0
:1060D0002448FFF731FF2448FFF722FF2348FFF74A
:1060E0002BFF2348FFF71CFF05E02248FFF718FFAE
:1060F0000135202D1AD0606C00EB8500FFF71CFFE6
:1061000005F00302032A1B4808BF1B48FFF708FFDE
:10611000616C013501EB8500FFF70EFF05F003030D
:10612000032BE2D11448FFF7FBFEE1E71248FFF72B
:10613000F7FEFEE70830002010850020A89902082D
:10614000D8990208E0990208E8990208F099020833
:10615000FC990208049A0208109A0208189A020888
:10616000209A02082CED00E02C9A020828ED00E0AD
:10617000389A0208D4990208449A0208024BEFF3B5
:1061800008825A6452E700BF10850020FEE700BF76
:10619000FEE700BFFEE700BFDEF732B8DEF732B839
:1061A00038B5444C1320A36C00215A1CA264DEF7BE
:1061B0004DF8B4F84C0083B223B1B4F84C00411E42
:1061C000A4F84C1094F84E203A4B002A4BD11422DC
:1061D00083F84E201D6D15B1186D411E1965B4F878
:1061E00054E0344B1FFA8EFCBCF1130F41D9B3F8C5
:1061F0005450143DA3F8545094F856302D4D312B83
:1062000040D895F856104A1C85F8562094F85C1032
:10621000284B4A1C84F85C2094F85CE0BEF10B0F1C
:106220000ED9002283F85C2093F85DE0DEF1010CCA
:1062300038BF4FF0000C012083F85DC083F85E008A
:1062400094F85F101B4B21B193F85F20501E83F828
:106250005F0094F86010174B21B193F86020501E36
:1062600083F8600038BD93F84E00411E83F84E104D
:1062700038BD03200021DDF7E9FF94F856300D4DBD
:10628000312BBED90023042085F856300121DDF7DB
:10629000DDFFB5F85820531CA5F85830B5F85AC0A2
:1062A0001FFA8CF00028B1D0B5F85A00411EA5F8AD
:1062B0005A10ABE71085002040F6D87320F000425A
:1062C000C3F6497301469A4200B583B015DDB2F1B9
:1062D000FF4F03DB02F026FF03B000BD694600F06C
:1062E000E9FF00F00302012A12D0022A09D0B2B954
:1062F0000098019901F0E2F9EEE7002101F0DEF9E2
:10630000EAE70098019901F0D9F900F10040E3E7CC
:106310000098019901F0CCFD00F10040DCE7009805
:106320000122019901F0C4FDD6E700BFD0F10103BD
:1063300038BF0023B0F1004F08BF43F00103002B2A
:106340002ED1A0F5000300F1FF42B3F1FE4F2CBFA8
:1063500000230123B2F1FE4F38BF43F00103EBB934
:106360004FF6FE73411EC0F27F0300F10042013A76
:1063700099428CBF002101219A428CBF0B4641F00B
:1063800001037BB910F5000F14BF00230123B0F106
:10639000FF4F14BF184643F00100704704207047B8
:1063A000022070470320704740F6D87320F0004267
:1063B000C3F6497301469A4200B583B016DDB2F1C7
:1063C000FF4F03DB02F0AEFE03B000BD694600F0F4
:1063D00071FF00F00300012815D002280BD0B8B9D6
:1063E00000980122019901F063FDEDE700210022F0
:1063F00001F05EFDE8E700980122019901F058FDE7
:1064000000F10040E0E70098019901F057F9DBE75F
:106410000098019901F052F900F10040D4E700BF63
:1064200000F080BA70B58AB0054600F031FB43F247
:106430000C04C2F2000494F90030B3F1FF3F0646A9
:106440003AD02846FFF772FF002835D028460021B1
:1064500003F01AF900282FD049F648232846C0F641
:10646000020301930023089302F01AFB24780246EA
:106470000B46CDE90423CDE90223002C1FD00023D5
:10648000284600210022CFF6F073CDE9062303F061
:10649000E7F8002821D0022300939C4233D06846BD
:1064A00001F086FD00282ED0089B002B26D1DDE9C7
:1064B000060102F0E3FD064630460AB070BD4FF615
:1064C000FF73284600214FF06042CCF2EF73CDE914
:1064D000062303F0C5F80028DDD10123022C009328
:1064E00016D0684601F064FD90B149F6A000C0F6F0
:1064F000020001F05FFDCDE90601D5E703F028F9C0
:10650000089B0360D3E703F023F922230360CBE762
:1065100003F01EF921230360E7E700BF2DE9F041F6
:106520008AB007460D4600F00DFB43F20C06C2F29E
:10653000000696F90030B3F1FF3F044603D0284629
:10654000FFF7F4FE18B920460AB0BDE8F0813846DE
:10655000FFF7ECFE8046002832D12846002103F0E8
:106560007FF80028EFD049F650233846C0F60203E2
:10657000CDF8208001930123009302F091FACDE938
:106580000201284602F08CFA96F90040002300220E
:10659000C3F6F073CDE90623A4F1FF32534243EB77
:1065A0000203022C14BF1C4643F00104CDE9040190
:1065B000002C32D0DDE9060102F060FD0446C2E79E
:1065C0003846002103F04CF8002833D0284600213B
:1065D00003F046F800286AD049F650233846C0F642
:1065E00002030193012300930023089302F058FA59
:1065F000CDE90201284602F053FA96F90040002244
:106600000023CDE90623CDE9040134B100230022A3
:10661000C3F6F073CDE90623CCE7684601F0C8FC69
:10662000002874D0089B002BC4D003F091F8089B7D
:106630000360BFE7204601F087FE804600286BD04C
:106640002046002103F00CF800283FF47CAF3846C8
:1066500001F07AFE00283FF476AF284601F074FE80
:1066600000283FF470AF49F650233846C0F60203C5
:106670000193042300930023089302F011FACDE95B
:106680000201284602F00CFA96F90040002200238D
:10669000022CCDE90623CDE9040176D0684601F04D
:1066A00087FC002871D0089B002B83D0BDE72846CB
:1066B00001F04AFE00283FF446AF2846002102F0D0
:1066C000D9FF00283FF43FAF49F650233846C0F6C3
:1066D00002030193012300930023089302F0E0F9E1
:1066E000CDE90201284602F0DBF93478CDE9040156
:1066F000002C45D000220023022CCFF6F073CDE908
:10670000062337D103F024F821230360CBE703F0FD
:106710001FF82123036085E7384601F015FE0028A5
:106720008ED0284601F010FE002889D02046FFF7C1
:10673000FDFD024600282DD149F650233846C0F60B
:106740000203089201930123009302F0A9F9CDE915
:106750000201284602F0A4F93478CDE904017CB1A5
:106760000020002102460B4602F018FB022CCDE966
:106770000601C7D0684601F01BFC002893D1C1E791
:1067800000220023CDE90623F4E702F0E1FF2223F3
:10679000036088E749F650233846C0F60203CDF877
:1067A000208001930323009302F07AF9CDE90201DE
:1067B000284602F075F996F90030CDE90401E3B9F5
:1067C0004FF6FF73384600214FF06042C4F2EF737A
:1067D000CDE9062302F04EFF002834D196F90030AF
:1067E000022B05D0684601F0E3FB00287FF41AAFC6
:1067F00002F0AEFF2223036014E700233846002195
:106800000022C7F6F073CDE9062302F033FF00281B
:10681000E4D04FF07C51284602F08EFD02F040F9A2
:1068200004460D4601F0CCFB02460B4620462946A5
:1068300002F0F2FB0028D1D100230022CFF6F07342
:10684000CDE90623CAE74FF07C51284602F074FDDB
:1068500002F026F904460D4601F0B2FB02460B4653
:106860002046294602F0D8FB0028B7D14FF6FF7327
:106870004FF06042CCF2EF73CDE90623AEE700BFE4
:1068800070B58AB0064600F0C1FE43F20C04C2F2B5
:10689000000494F90030B3F1FF3F054630D0304694
:1068A000FFF744FD00282BD03046002102F0E2FE25
:1068B00030B349F658233046C0F602030193012352
:1068C00000930023089302F0EBF82478CDE904014B
:1068D000CDE90201BCB10020002102460B4602F0C6
:1068E0005DFA022CCDE9060111D102F031FF21231E
:1068F0000360089B8BB9DDE9060102F0BFFB05468A
:1069000028460AB070BD00220023CDE90623684660
:1069100001F04EFB0028ECD1E7E702F019FF089BDD
:106920000360E8E72DE9F04120F00044B4F1FF4FA7
:1069300021F00046D4BF00270127B6F1FF4FC8BFA2
:1069400047F001070346002F49D1B1F17E5F51D0D6
:106950008F1707F0020747EAD07754B9022F44D0C7
:10696000032F03D140F6DB73CCF249031846BDE890
:10697000F08136B3B6F1FF4F59D0B4F1FF4F20D0BC
:10698000A41BE4153C2CC4BF40F6DB70C3F6C970F1
:1069900034DD012F08BF00F10043E7D0022F37D0CC
:1069A0000346002FE2D04BF62E51C3F2BB3102F06A
:1069B000BBFB40F6DB71C4F2490102F0B3FB0346B6
:1069C000D4E70028BCBF40F6DB73CBF6C973CDDB40
:1069D00040F6DB73C3F6C9731846BDE8F08102F0D8
:1069E000A3FB03461846BDE8F08140F6DB73C4F212
:1069F0004903BBE7BDE8F04101F080BB14F13C0F57
:106A0000ACBF0024012414EAD1741ED00020C0E7DA
:106A10004BF62E51C3F2BB3102F086FB014640F625
:106A2000DB70C4F2490002F07DFB03469EE7B4F13F
:106A3000FF4F11D0022FD8D0032F93D0012F08BFC2
:106A40004FF0004392D0002390E702F029FD01F0BF
:106A500077FC01F053FB9CE7022F04BF4CF6E433B4
:106A6000C4F2160382D0032F04BF4CF6E433CCF2F9
:106A700016033FF47BAF012F1CBF40F6DB73C3F658
:106A800049737FF473AF40F6DB73CBF649736DE760
:106A900020F00043014670B50646002B43D0002885
:106AA00047DBB0F1FF4F4ADAB0F5000FA8BF6FF037
:106AB0007E0006DA4FF0984102F03EFC06466FF089
:106AC000970000EBE65026F07F4626F40006C50F3F
:106AD000281802F0DDFB0446C5F17F0046EAC050ED
:106AE00001F0EEFC4FF40251C3F69A6106462046CF
:106AF00002F022FC42F2DB71C3F2545105462046FB
:106B000002F01AFC45F6D931C3F6DE610446304680
:106B100002F012FC0146204602F006FB0146284620
:106B200002F002FB70BD00214FF04C4002F0B8FCB7
:106B300070BD02F0F7FA002102F0B2FC70BD02F065
:106B4000F3FA70BD2DE9F04F31F0004987B00C46E3
:106B500082460D464BD020F000478046B7F1FF4FEC
:106B6000D4BF00260126B9F1FF4FC8BF46F0010689
:106B7000002E39D1002864DBB9F1FF4F46D0B9F1BE
:106B80007E5F4AD0B5F1804F00F0A180B5F17C5F07
:106B900002D1B8F1000F72DA504601F0D1FBA7F133
:106BA000FF42534243EB0203002F08BF43F00103AF
:106BB0000146002B3CD1B7F17E5F39D04FEAD8783F
:106BC00008F1FF3856EA080100F08780B9F19A4FC2
:106BD00040F394804FF6F773C3F67F739F4265DCF2
:106BE000002D6BDB002404E0B7F17E5F05D14FF090
:106BF0007E54204607B0BDE8F08F49F6A000C0F6ED
:106C0000020007B0BDE8F04F01F0F6BBB7F17E5FC0
:106C1000EDD02DDD002DECDAE4E7002DA8BF5446C1
:106C2000E7DA4FF07E50514602F03AFC0446E0E7C6
:106C3000002DA8BF084634DBB8F1000F25DB044661
:106C4000D7E7B9F1974F11DAB9F17E5F97DB4FEAD9
:106C5000E953C3F1960349FA03F212FA03F34B45E1
:106C600004BF02F00102C2F1020688E7022683E7B0
:106C7000002DB8BF04F10044BBDB0024B9E7504647
:106C800007B0BDE8F04F00F0C1BCA7F17E57374315
:106C90002CD1014602F046FA014602F001FC0446FE
:106CA000A7E74FF07E5002F0FBFBC5E70723C3F6D2
:106CB00080739F4240F3AD82002D93DD4FF2CA20D6
:106CC000C7F24910014602F037FB044691E75046EF
:106CD000514602F031FB04468BE75146504602F024
:106CE00021FA014602F0DCFB044682E7012E08BFD0
:106CF00000F100443FF47DAF04467AE7B7F5000F9A
:106D0000A8BF6FF07E0106DA4FF0974102F014FB46
:106D10006FF09601074627F07F434CF2714223F44F
:106D20000003C0F21C02934201EBE75143F07E578F
:106D3000049140F300824BF2D632C0F25D029342DE
:106D400040F3AE82A7F50007002201314FF4802303
:106D50000491059349F660233846C0F60203BA460B
:106D600003EB8201039153F822B0594602F0DAF99D
:106D700039460290584602F0D7F901464FF07E504E
:106D800002F08EFB024602981146009202F0D4FAFD
:106D90007B10059943F000535B1801931946814617
:106DA00020F47E6020F01F00074602F0C5FA01467D
:106DB000029802F0B7F9019B594684461846CDF86F
:106DC00004C002F0AFF90146504602F0ABF9394673
:106DD00002F0B2FADDF804C00146604602F0A2F902
:106DE000009A114602F0A8FA49468346484602F046
:106DF000A3FA0146824602F09FFA4FF24211C3F60F
:106E0000536103465046019302F096FA43F255212E
:106E1000C3F66C6102F088F9514602F08DFA4AF22D
:106E20000531C3F68B6102F07FF9514602F084FA16
:106E30004AF6AB21C3F6AA6102F076F9514602F098
:106E40007BFA46F6B751C3F6DB6102F06DF95146A5
:106E500002F072FA49F69A11C3F6197102F064F958
:106E6000019B0146184602F067FA394682464846B9
:106E700002F05AF9594602F05FFA514602F054F90D
:106E800039460290384602F057FA0021C4F2400118
:106E9000019002F049F9029902F046F920F47E6A65
:106EA00038462AF01F0A514602F046FA5146074674
:106EB000584602F041FA0021C4F240018346504690
:106EC00002F030F9019B194602F02CF901460298B4
:106ED00002F028F9494602F02FFA0146584602F01E
:106EE00023F983463846594602F01EF94FF46051A3
:106EF000C3F6767120F47E6929F01F09484602F036
:106F00001BFA4CF2A031C3F29D618246484602F062
:106F100013FA394603464846019302F003F9014645
:106F2000584602F0FFF843F64F01C3F6767102F0BF
:106F300003FA019B0146184602F0F6F8039B996894
:106F400002F0F2F80746049802F0A2F939468146A9
:106F50000398D0F810B0504602F0E6F8594602F017
:106F6000E3F8494602F0E0F8494620F47E6929F04A
:106F70001F09484602F0D6F8594602F0D3F85146A8
:106F800002F0D0F8013E0146384602F0CBF856EA4E
:106F9000080618BF4FF07E56074602D10026CBF6F2
:106FA000807625F47E65204625F01F05294602F0EF
:106FB000B9F8494602F0C0F939468046204602F049
:106FC000BBF90146404602F0AFF8294680464846E4
:106FD00002F0B2F9054601464046AA4602F0A4F87E
:106FE000002807460446034620F0004940F3F3809A
:106FF000B9F1864F00F3B58000F0A280B9F17C5F53
:10700000DCBF4FF000094F4600F3BA8023F47E64E2
:107010004FF4E44124F01F04C3F63171204602F01E
:107020008BF951460546204602F07CF80146404661
:1070300002F078F847F21821C3F6317102F07CF9BA
:107040004BF68C61C3F2BF518046204602F074F9C2
:107050000146404602F068F880462846414602F064
:1070600063F82946044602F05DF80146404602F006
:1070700059F821468046204602F05EF94BF64C3125
:10708000C3F23131054602F057F94EF60E21C3F234
:10709000DD5102F047F8294602F04EF94BF2553126
:1070A000C3F68A0102F040F8294602F045F940F69D
:1070B0006131C3F6363102F035F8294602F03CF969
:1070C0004AF6AB21C3F62A6102F02EF8294602F0F7
:1070D00033F90146204602F025F8054620462946A8
:1070E00002F02AF94FF080418246284602F01AF851
:1070F0000146504602F0D4F941460546204602F0CA
:107100001BF9414602F010F80146284602F00AF841
:10711000214602F007F801464FF07E5002F002F8D7
:1071200000EB0901CB15002B40F3BF80304602F085
:1071300003F904465DE54FF480200022059009E63E
:107140004AF63C214046C3F2383101F0EDFF2946B2
:107150008246384601F0E6FF0146504602F0A8FAA2
:1071600070B14FF2CA213046C7F2491102F0E4F87B
:107170004FF2CA21C7F2491102F0DEF8044638E5A1
:107180004FEAE9534FF400027F3B4FF6FF710133A2
:10719000C0F27F0152FA03F328461B1923F07F4700
:1071A000C3F3C75227F400077F3A47F400071141A1
:1071B000C2F1170223EA01011741002CB8BF7F4238
:1071C00001F0B0FF4FEAC75982464046514601F0F0
:1071D000ABFF03461AE70022C4F21632914509DCE0
:1071E0007FF40CAF294601F09DFF414602F056FAAC
:1071F0000028C5D044F260213046C0F6A25102F00A
:107200009BF844F26021C0F6A25102F095F80446C2
:10721000EFE44FF07E5101F085FF4FF42A41C3F6B1
:10722000B871074602F088F84AF27051C3F2EC6177
:107230008146384602F080F839468246384602F0E8
:107240007BF84FF07A518346384602F075F80146D4
:107250004AF6AB20C3F6AA6001F064FF394602F09B
:107260006BF801464FF07C5001F05CFF0146584638
:1072700002F062F84AF63B21C3F6B87102F05CF8FE
:107280000146504601F04EFF07464846394601F098
:107290004BFF494620F47E6929F01F0948466FE6F6
:1072A0004FF410110122059154E5394601F0A8F878
:1072B00001463BE740F6D8732DE9F04FC3F649731A
:1072C00020F0004687B09E4205460C4640F38E8073
:1072D0004CF6E333C4F216039E4226DC002840F34A
:1072E0004E814FF4786126F00F06C3F6C97101F0A4
:1072F00019FF4FF47D63C3F6C9739E42054600F043
:10730000848044F243410127C3F2357101F00AFF42
:1073100001462060284601F005FF44F24341C3F2D4
:10732000357101F0FFFE606064E04FF47863C4F2F1
:1073300049339E4240F38480B6F1FF4F5EDA4FEA54
:10734000E659A9F186094FEAC953F61A304602F008
:10735000B9F901F09DFF034601463046039301F061
:10736000E1FE4FF0874101F0E7FF064602F0AAF97F
:1073700001F08EFF014607463046049701F0D2FE29
:107380004FF0874101F0D8FF0021059002F068F925
:10739000002800F018810DF10C0A03263846002160
:1073A0000AF10408013E02F05BF940B158F8047D8F
:1073B0000021013E384602F053F90028F6D1334649
:1073C000914E504621464A4601960226009600F00C
:1073D00051FA002D07460DDA22684742636802F130
:1073E0000042226003F10043636003E000270023B2
:1073F00008604B60384607B0BDE8F08F01460027B3
:1074000001F090FE60602060F4E74FF488410127AE
:10741000C3F2357101F086FE4AF20831C2F6856189
:10742000054601F07FFE01462060284601F07AFE05
:107430004AF20831C2F6856101F074FE6060D9E756
:1074400000F07EFF4FF68411C3F62271804601F0F2
:1074500073FF4FF07C5101F067FE02F033F90746ED
:1074600001F016FF4FF47861C3F6C971824601F04E
:1074700063FF0146404601F055FE44F24341C3F22A
:1074800035718046504601F057FF1F2F81461CDCA6
:1074900049F67823791EC0F6020326F0FF0253F85E
:1074A00021309A4211D04946404601F03BFE014648
:1074B0002060404601F036FE494601F033FE002DC3
:1074C000606097DA22687F4288E74946404601F0CB
:1074D00029FEF615C0F3C7530146F31A2060082BA6
:1074E000E7DD4FF488415046C3F2357101F024FFC7
:1074F00081464046494601F015FE834640465946BE
:1075000001F010FE494601F00DFE4AF20831C2F6C4
:1075100085618046504601F00FFF414601F002FEB2
:1075200081465846494601F0FDFDC0F3C753014668
:10753000F61A2060192ED8BFD846BADD4FF4234181
:107540005046C2F6856101F0F7FE064658463146C0
:1075500001F0E8FD80465846414601F0E3FD314622
:1075600001F0E0FD43F23211C2F28D410646504671
:1075700001F0E2FE314601F0D5FD814693E74FF47C
:10758000786126F00F06C3F6C97101F0CDFD4FF406
:107590007D63C3F6C9739E42054618D044F2434149
:1075A0004FF0FF37C3F2357101F0BEFD0146206098
:1075B000284601F0B7FD44F24341C3F2357101F0B2
:1075C000B3FD606016E703260DF10C0AF7E64FF4F1
:1075D00088414FF0FF37C3F2357101F0A5FD4AF243
:1075E0000831C2F68561054601F09EFD0146206026
:1075F000284601F097FD4AF20831C2F6856101F094
:1076000093FD6060F6E600BFF89A020820F00042A1
:107610000346B2F1FF4F70B504463AD2002A36D085
:10762000002840DBC115B2F5000F09D210F40002AA
:1076300041D15B00013213F4000FFAD00131891AF5
:1076400023F07F43A1F17F0223F4000312F0010F26
:1076500043F4000318BF5B000026541019215B009F
:1076600035464FF08072A8189842DEBFC0EB030386
:107670008518B61852085B000139F4D113B106F031
:1076800001039E19E40504F17C5404EB66042046D2
:1076900070BD014601F050FE0146204601F044FD58
:1076A0000446204670BD014601F03CFD014601F054
:1076B000F7FE0446EBE70022C0E700BF2DE9F843E0
:1076C00020F00046B6F1485F05460F465BDA01F050
:1076D000F9FF002800F0CA802946284601F02CFE58
:1076E0004DF24E71CAF64751044601F025FE47F2AD
:1076F000F641C3F20F1101F017FD214601F01CFE07
:107700004FF27C21C3F2934101F00CFD214601F0C0
:1077100013FE40F60151C3F2D07101F005FD214680
:1077200001F00AFE40F66131C3F6B62101F0FAFC21
:10773000214601F001FE4AF6AB21C3F62A5101F0C1
:10774000F3FC214601F0F8FD804620464FF07C51C5
:1077500001F0F2FD41460646204601F0EDFD3946B6
:107760000446284601F0E8FD0146204601F0DAFC17
:107770000146304601F0D6FC01464FF07E5001F044
:10778000D1FCBDE8F883014601F0D6FD4DF24E7103
:10779000CAF64751044601F0CFFD47F2F641C3F265
:1077A0000F1101F0C1FC214601F0C6FD4FF27C2112
:1077B000C3F2934101F0B6FC214601F0BDFD40F655
:1077C0000151C3F2D07101F0AFFC214601F0B4FDCC
:1077D00040F66131C3F6B62101F0A4FC214601F068
:1077E000ABFD4AF6AB21C3F62A5101F09DFC2146C0
:1077F00001F0A2FD49F69913C3F699639E428046B3
:10780000A3DD0023C3F648739E4227DC06F17F46C2
:107810004FF07E50314601F085FC814620464FF006
:107820007C5101F089FD314601F07CFC4146064661
:10783000204601F081FD39460446284601F07CFDD2
:107840000146204601F06EFC0146304601F06AFC1C
:107850000146484601F066FCBDE8F8834FF0000998
:107860000026C3F63879C3F69066D7E74FF07E500E
:10787000BDE8F8832DE9F04FDDB049F610651C46F0
:107880000791013B6699C0F602050193D31E48BFDC
:10789000131D039055F82150DB1023EAE37308937E
:1078A000DB430695069902EBC303019A049311EB9F
:1078B00002081BD4089B33AF67999D1AA84401EBBB
:1078C000850609E03068043601F0E2FC454505F123
:1078D000010547F8040F09D0002DF3DA0020043623
:1078E000454547F8040F05F10105F5D1069A002A30
:1078F000C0F2CC82069A0CA9A1460DF12C0A059182
:1079000001EB820B019B002BC0F25F8134A9DDF8F3
:107910000C8001EB89070026002557F8041D01356E
:1079200058F8040B01F008FD0146304601F0FCFB5D
:10793000A5420646F1D14AF8046FDA4509F101097A
:10794000E0D1069A48A9531E924601EB82015CAA37
:107950009B000A91D21809930B92059BBAF1000F74
:1079600053F82A5022DD48A903EB8A060F1F9946D7
:107970004FF06E51284601F0DFFC01F0A3FE01F04C
:1079800087FC4FF08741804601F0D6FC014628462F
:1079900001F0C8FB01F096FE414647F8040F56F887
:1079A000040D01F0C1FB4E450546E1D1049928467E
:1079B00000F026FD4FF07851054601F0BDFC00F0C7
:1079C000CBFC4FF0824101F0B7FC0146284601F0A4
:1079D000A9FB054601F076FE074601F059FC014679
:1079E000284601F09FFB049A002A064640F3D08007
:1079F0000AF1FF33C2F10801C2F107055CAA02EBEC
:107A0000830353F8502C52FA01F03F1810FA01F199
:107A1000521A43F8502C42FA05FBBBF1000F32DD3D
:107A20000137BAF1000F40F32F8248AB002503EB7A
:107A30008A0107E022B10125C2F5807243F8042CC7
:107A40008B420AD053F8042B002DF3D001258B4232
:107A5000C2F1FF0243F8042CF4D1049A002A0FDD8E
:107A6000012A00F09E80022A0AD10AF1FF335CAAA3
:107A700002EB830353F8502C02F03F0243F8502CE2
:107A8000BBF1020F71D03046002101F0E9FD002862
:107A900000F0A080069B9A450DDD48A90A9801EBED
:107AA0008A03002253F8041D834242EA0102F9D1FD
:107AB000002A40F0C6800B9A52F8503C002B40F050
:107AC000E181099B48A9CA18012352F8041D01331A
:107AD0000029FAD053440AF101099945029338DC90
:107AE000089A0AEB04036799013B0AEB020B059A1B
:107AF00002EB8A0A01EB8B0B34A901EB83010091A5
:107B00005BF8040F01F0C4FB019B009A002B42F8C4
:107B1000040F009220DB09EB040734A9DDF80C8088
:107B20000026002501EB870757F8041D013558F89A
:107B3000040B01F001FC0146304601F0F5FAA542C4
:107B40000646F1D1029A09F101094AF8046F9145FC
:107B5000D6DDDDF808A000E7029A09F10109002648
:107B60004AF8046F9145CBDDF3E731464FF07E5084
:107B700001F0D8FA0646002D85D004994FF07E50CA
:107B800000F03EFC0146304601F0CCFA06467AE7AA
:107B900013D15CA901EB8A0353F8543C4FEA232B21
:107BA0003BE70AF1FF335CA901EB830353F8502C48
:107BB00002F07F0243F8502C62E74FF07C5101F055
:107BC0006DFD20B94FF0000B5DE70026B3E64FF0E6
:107BD000020B25E70097002834D1049A3046514221
:107BE00000F00EFC4FF08741044601F057FD0028DD
:107BF00000F04F814FF06E51204601F09DFB5CABD1
:107C000003EB8A0501F05EFD01F042FB0AF1010A77
:107C10005CAA4FF0874102EB8A07064601F08CFB15
:107C20000146204601F07EFA049B0833049301F0DC
:107C300049FD45F8500C304601F044FD47F8500C22
:107C400017E00097049B0AF1FF3A5CAC083B0493F1
:107C50004FEA8A03E21852F8502C52B948A9049A04
:107C6000CB1853F8041D0AF1FF3A083A0029F8D05E
:107C700004924FF07E50049900F0C2FBBAF1000F5D
:107C800005464CDB0AF10106059A48AFB600BC195F
:107C9000961954F8040D01F0FBFA294601F04CFB4B
:107CA0004FF06E5146F8040D284601F045FBBC42EA
:107CB0000546EED10AF1FF39CDF804A0DDF818A091
:107CC0004FF00008BAF1000FC0F2D880B8F1000FF1
:107CD000C0F2D48005990025744F002401EB890679
:107CE00001E044450DDC56F8041F013457F8040F39
:107CF00001F022FB0146284601F016FAA24505468E
:107D0000EFDA5CAC09F1FF3904EB880319F1020FDB
:107D100008F1010843F8F05CD4D1DDF804A0669ABC
:107D2000032A13D8DFE802F0936565180020BBF141
:107D3000000F57D0079900F10040219B209A03F1D2
:107D40000043886002F100424B600A60009A02F032
:107D500007005DB0BDE8F08FBAF1000FE6DD20ADA1
:107D600005EB8A0454F8048C54F8047940463946EB
:107D700001F0DAF906464046314601F0D3F90146F2
:107D8000384601F0D1F9AC4226606060EAD1BAF120
:107D9000010FCBDD0AF1FF3405EB840454F80489AC
:107DA0004046A768394601F0BFF9064640463146CD
:107DB00001F0B8F90146384601F0B6F9AC42666008
:107DC000A060EBD10AF1010A04F10805002004EBE0
:107DD0008A0454F8041D01F0A7F9AC42F9D1BBF1B3
:107DE000000FA7D1209A219B079CA06022606360AE
:107DF000ACE7BAF1000F57DB0AF1010420AD002017
:107E000005EB840454F8041D01F08EF9AC42F9D15D
:107E1000BBF1000F34D000F1004307990B6001461D
:107E2000209801F07FF9BAF1000F08DD20AC04EBD7
:107E30008A0A54F8041F01F077F95445F9D1BBF1CF
:107E4000000F01D000F10040079A50607EE7BAF1C0
:107E5000000F27DB0AF1010420AD002005EB8404AC
:107E600054F8041D01F060F9AC42F9D1BBF1000FE8
:107E700001D000F10040079C206067E7002540E743
:107E80000346CAE7012325E60025E6E50CAB05938A
:107E900057E520465CA901EB8A0401F013FC44F885
:107EA000500CE6E60020E1E70020B1E7189E02084A
:107EB0002DE9F84320F00043B3F1485F04460D4636
:107EC000904603DA01F0FEFB002859D021462046F7
:107ED00001F032FA2146064601F02EFA4CF6D31193
:107EE000C2F62E710746304601F026FA42F634718A
:107EF000C3F2D72101F016F9314601F01DFA4EF612
:107F00001B71C3F2386101F00FF9314601F014FA28
:107F100040F60151C3F6501101F004F9314601F069
:107F20000BFA48F68901C3F6084101F0FDF88146D5
:107F3000B8F1000F27D028464FF07C5101F0FCF932
:107F400049468046384601F0F7F90146404601F0BF
:107F5000E9F8314601F0F0F9294601F0E3F84AF674
:107F6000AB21C3F62A610546384601F0E5F9014622
:107F7000284601F0D9F80146204601F0D3F804461E
:107F80002046BDE8F8830146304601F0D5F94AF6AF
:107F9000AB21C3F62A6101F0C5F8394601F0CCF9EE
:107FA0000146204601F0C0F804462046BDE8F883AB
:107FB0000020704700210020C7F6F871704700BF0D
:107FC0002DE9F041C1F30A58A8F57E78CD0FA8F14C
:107FD000070C82B0BCF1130F02460B4604460F4655
:107FE0000E463DDCBCF1000F59DB4FF6FF71C0F2CD
:107FF0000F0141FA0CF101EA030010432BD04908AC
:1080000001EA030353EA02040DD04FF4802327EA68
:108010000106BCF1130F0CBF4FF00044002443FADB
:108020000CFC46EA0C0649F648612246C0F60201FD
:10803000334601EBC505D5E900452046294600F049
:10804000D1FB22462B46CDE90001DDE9000100F01D
:10805000C7FB02460B461046194602B0BDE8F08148
:10806000BCF1330F07DDBCF5806FF4D100F0BAFB33
:1080700002460B46EFE74FF0FF31A8F11B0821FA4B
:1080800008F10142E7D0490801421FBF4FF0804389
:1080900020EA010443FA08F844EA0804C3E721F09F
:1080A00000410143D7D023F07F4049F6486120F4D6
:1080B0007000C0F6020140EA020401EBC501604213
:1080C0004FEA534E40EA0404D1E90067240B3046DE
:1080D00004F40024394644EA4E4300F083FB324660
:1080E0003B46CDE90001DDE9000100F079FB21F01C
:1080F0000041024641EAC573ADE700BF2DE9F041FA
:1081000020F00045B5F1A14F044606460EDBB5F15F
:10811000FF4F00F3A5800028C4BF40F6DB74C3F610
:10812000C97440F3DA802046BDE8F0814FF6FF7352
:10813000C3F6DF639D4200F3A880B5F1445FC0F24F
:1081400096804FF0FF372146204601F0F5F80146B2
:10815000804601F0F1F846F6D711C3F68541054691
:1081600001F0EAF84DF65921C3F64B5100F0DCFF5F
:10817000294601F0E1F846F63531C3F6885100F0A2
:10818000D3FF294601F0D8F842F66E61C3F6BA5122
:1081900000F0CAFF294601F0CFF844F62511C3F6D6
:1081A000126100F0C1FF294601F0C6F84AF6AB2182
:1081B000C3F6AA6100F0B8FF414601F0BDF84AF2EB
:1081C0002121CBF615518046284601F0B5F84FF233
:1081D0006B11C3F66E5100F0A5FF294601F0ACF813
:1081E00048F29571C3F69D5100F09CFF294601F0BD
:1081F000A3F848F63861C3F6E35100F093FF29462F
:1082000001F09AF84CF6CD41C3F64C6100F08AFFBC
:10821000294601F091F8B7F1FF3F014651D049F6E8
:108220005865404600F080FFC0F60205214601F087
:1082300083F805EB8703196900F074FF214600F00D
:1082400071FF014655F8270000F06CFF002EB8BF03
:1082500000F10044FFF667AF04462046BDE8F08118
:10826000014600F061FF04462046BDE8F0814FF270
:10827000CA21C7F2491100F057FF4FF07E5101F0BB
:1082800017FA00283FF45DAF4DE700F059F84FF6BC
:10829000FF73C3F697739D42044623DC4FF6FF73CA
:1082A000C3F62F739D4241DC0146002700F03CFFDE
:1082B0004FF07E5100F036FF4FF0804105462046DA
:1082C00023E0404600F030FF214601F035F801463A
:1082D000204600F027FF044625E740F6DB74CBF686
:1082E000C97420E74FF6FF73C4F21B039D4214DCF0
:1082F0004FF07F51022700F015FF4FF07F510546E8
:10830000204601F019F84FF07E5100F00DFF0146B4
:10831000284601F0C5F8044615E700202146CBF6B3
:108320008070032701F0BCF804460CE74FF07E5143
:10833000012700F0F7FE4FF07E5105462046E4E7A6
:1083400020F00040704700BF20F00040B0F1FF4F28
:10835000ACBF0020012070472DE9F04120F000461D
:1083600001460446F50D7F3D162D1ADC002D804692
:1083700020DB4FF6FF77C0F27F072F4107420DD079
:108380004FF2CA21C7F2491100F0CEFE002101F0E0
:108390008FF9E8B1002C1FDB28EA07010846BDE889
:1083A000F081B6F1FF4FF9D300F0BEFE014608465A
:1083B000BDE8F0814FF2CA21C7F2491100F0B4FEC6
:1083C000002101F075F918B1002C0EDB0021E5E762
:1083D00021460846BDE8F0814FF4000353FA05F545
:1083E00004EB050828EA0701D8E70021CBF68071E5
:1083F000002E08BF2146D1E70020C7F6C0707047A5
:1084000010B50C4630F000410346024625D0B1F1CC
:10841000FF4F24D2B1F5000F27D3C90D0919FE294A
:1084200033DC0029C4BF22F0FF4242EAC15314DC0E
:1084300011F1160F38DA4CF25032944225DC44F236
:1084400060201946C0F6A25000F0BEF944F2602147
:10845000C0F6A25100F070FF0346184610BD014659
:1084600000F062FE0346184610BD4FF0984100F040
:1084700063FF43F6B042CFF6FF7294420346E5DB5A
:10848000C0F3C75102461939C8E74FF2CA2019464E
:10849000C7F2491000F098F94FF2CA21C7F249110A
:1084A00000F04AFF0346D8E701F1190022F0FF422D
:1084B0004FF04C5142EAC05000F03EFF0346CCE77B
:1084C0002DE9F84F20F0004301460246002B00F052
:1084D000B3800028C0F2D680B0F1FF4F80F2CE808A
:1084E000B0F5000FA8BF6FF07E0706DA4FF0984195
:1084F0006FF0970700F020FF024622F07F444FF60E
:10850000203324F40004C0F24A03E31807EBE257D7
:1085100003F400034FF07E5183F07E50204307EBBD
:10852000D35700F0FFFD04F10F0323F400030F2BDA
:10853000054640F388804FF0804145F6304800F012
:10854000F3FDCFF6CF78A0440146284600F0A8FFFF
:108550008146384600F09CFE49468346484600F076
:10856000EBFE0146824600F0E7FE48F69701C3F6AF
:108570001761064600F0E0FE43F22531C3F63A618A
:1085800000F0D2FD314600F0D7FE44F62511C3F6C7
:10859000926100F0C9FD314600F0CEFE4AF6AB21F3
:1085A000C3F62A7100F0C0FD514600F0C5FE4DF241
:1085B0004F01C3F61C618246304600F0BDFE48F60E
:1085C0002961C3F6636100F0AFFD314600F0B4FEEF
:1085D0004CF6CD41C3F6CC6100F0A6FD314600F06B
:1085E000ABFE0146504600F09FFD4CF28823C0F2DE
:1085F00035031B1B43EA0808B8F1000F064640F399
:10860000B0804FF07C51284600F096FE294600F0DD
:1086100093FE0446002F5AD1314600F085FD4946AD
:1086200000F08AFE0146204600F07CFD0146284607
:1086300000F078FDBDE8F88F00214FF04C4000F0CD
:108640002FFFBDE8F88F002101F00AF808B3002FD2
:1086500000F08480384600F01BFE4FF4E341C3F67F
:108660003171054600F068FE4FF2D171C3F2177107
:108670000446284600F060FE0146204600F054FD06
:10868000BDE8F88F00F04EFD002100F009FFBDE8C5
:10869000F88F2946284600F04FFE4AF6AB21C3F674
:1086A000AA610446284600F047FE01464FF07C5080
:1086B00000F038FD0146204600F03EFE0446002F43
:1086C0002DD12846214600F02DFDBDE8F88F4FF44E
:1086D000E3415846C3F6317100F02EFE314607469D
:1086E000204600F021FD494600F026FE4FF2D171F0
:1086F000C3F217710646584600F01EFE014630468A
:1087000000F012FD0146204600F00CFD294600F065
:1087100009FD0146384600F005FDBDE8F88F3846F2
:1087200000F0B6FD4FF4E341C3F63171074600F0A7
:1087300003FE4FF2D171C3F217710646384600F0BE
:10874000FBFD0146204600F0EDFC294600F0EAFC66
:108750000146304600F0E6FCBDE8F88F0020BDE899
:10876000F88F1FB34FF4E3415846C3F6317100F060
:10877000E3FD31460446284600F0D4FC494600F0AB
:10878000DBFD4FF2D171C3F217710646584600F077
:10879000D3FD0146304600F0C5FC294600F0C2FC7E
:1087A0000146204600F0BEFCBDE8F88F3146284661
:1087B00000F0B8FC494600F0BFFD0146284600F035
:1087C000B1FCBDE8F88F00BF01F0004120F000408F
:1087D00041EA0000704700BF81F0004102E000BFA5
:1087E00083F0004330B54FEA41044FEA430594EA71
:1087F000050F08BF90EA020F1FBF54EA000C55EAAC
:10880000020C7FEA645C7FEA655C00F0E2804FEA7C
:108810005454D4EB5555B8BF6D420CDD2C4480EA5E
:10882000020281EA030382EA000083EA010180EA8E
:10883000020281EA0303362D88BF30BD11F0004FDC
:108840004FEA01314FF4801C4CEA113102D0404212
:1088500061EB410113F0004F4FEA03334CEA13334D
:1088600002D0524263EB430394EA050F00F0A78065
:10887000A4F10104D5F1200E0DDB02FA0EFC22FA60
:1088800005F2801841F1000103FA0EF2801843FA54
:1088900005F359410EE0A5F120050EF1200E012A45
:1088A00003FA0EFC28BF4CF0020C43FA05F3C01883
:1088B00051EBE37101F0004507D54FF0000EDCF1FC
:1088C000000C7EEB00006EEB0101B1F5801F1BD3A5
:1088D000B1F5001F0CD349085FEA30004FEA3C0CA9
:1088E00004F101044FEA445212F5800F80F09A809F
:1088F000BCF1004F08BF5FEA500C50F1000041EBA3
:10890000045141EA050130BD5FEA4C0C404141EBA6
:10891000010111F4801FA4F10104E9D191F0000FCD
:1089200004BF01460020B1FA81F308BF2033A3F150
:108930000B03B3F120020CDA0C3208DD02F1140C47
:10894000C2F10C0201FA0CF021FA02F10CE002F182
:108950001402D8BFC2F1200C01FA02F120FA0CFC7B
:10896000DCBF41EA0C019040E41AA2BF01EB0451C4
:10897000294330BD6FEA04041F3C1CDA0C340EDCC2
:1089800004F11404C4F1200220FA04F001FA02F305
:1089900040EA030021FA04F345EA030130BDC4F1C3
:1089A0000C04C4F1200220FA02F001FA04F340EAB8
:1089B0000300294630BD21FA04F0294630BD94F069
:1089C000000F83F4801306BF81F480110134013D50
:1089D0004EE77FEA645C18BF7FEA655C29D094EAC1
:1089E000050F08BF90EA020F05D054EA000C04BF3F
:1089F0001946104630BD91EA030F1EBF002100202A
:108A000030BD5FEA545C05D14000494128BF41F0C8
:108A1000004130BD14F580043CBF01F5801130BD2C
:108A200001F0004545F0FE4141F470014FF00000B7
:108A300030BD7FEA645C1ABF194610467FEA655C68
:108A40001CBF0B46024650EA013406BF52EA03350A
:108A500091EA030F41F4002130BD00BF90F0000FF8
:108A600004BF0021704730B54FF4806404F1320434
:108A70004FF000054FF0000150E700BF90F0000FED
:108A800004BF0021704730B54FF4806404F1320414
:108A900010F0004548BF40424FF000013EE700BFE4
:108AA00042004FEAE2014FEA31014FEA02701FBF74
:108AB00012F07F4393F07F4F81F06051704792F046
:108AC000000F14BF93F07F4F704730B54FF46074C0
:108AD00001F0004521F0004120E700BF50EA01020B
:108AE00008BF704730B54FF000050AE050EA0102B8
:108AF00008BF704730B511F0004502D5404261EB28
:108B000041014FF4806404F132045FEA915C3FF468
:108B1000DCAE4FF003025FEADC0C18BF03325FEA01
:108B2000DC0C18BF033202EBDC02C2F1200300FAB6
:108B300003FC20FA02F001FA03FE40EA0E0021FADB
:108B400002F11444C1E600BF70B54FF0FF0C4CF4C5
:108B5000E06C1CEA11541DBF1CEA135594EA0C0F7B
:108B600095EA0C0F00F0DEF82C4481EA030621EAB6
:108B70004C5123EA4C5350EA013518BF52EA0335F1
:108B800041F4801143F4801338D0A0FB02CE4FF0A3
:108B90000005E1FB02E506F00042E0FB03E54FF0D3
:108BA0000006E1FB03569CF0000F18BF4EF0010ECB
:108BB000A4F1FF04B6F5007F64F5407404D25FEAC7
:108BC0004E0E6D4146EB060642EAC62141EA55517A
:108BD0004FEAC52040EA5E504FEACE2EB4F1FD0CBC
:108BE00088BFBCF5E06F1ED8BEF1004F08BF5FEA3A
:108BF000500E50F1000041EB045170BD06F00046EC
:108C000046EA010140EA020081EA0301B4EB5C0498
:108C1000C2BFD4EB0C0541EA045170BD41F4801190
:108C20004FF0000E013C00F3AB8014F1360FDEBFB5
:108C3000002001F0004170BDC4F10004203C35DA91
:108C40000C341BDC04F11404C4F1200500FA05F314
:108C500020FA04F001FA05F240EA020001F00042B5
:108C600021F0004110EBD37021FA04F642EB06012B
:108C70005EEA430E08BF20EAD37070BDC4F10C0455
:108C8000C4F1200500FA04F320FA05F001FA04F219
:108C900040EA020001F0004110EBD37041F1000105
:108CA0005EEA430E08BF20EAD37070BDC4F1200510
:108CB00000FA05F24EEA020E20FA04F301FA05F278
:108CC00043EA020321FA04F001F0004121FA04F220
:108CD00020EA020000EBD3705EEA430E08BF20EAF0
:108CE000D37070BD94F0000F0FD101F0004640002A
:108CF00041EB010111F4801F08BF013CF7D041EAAC
:108D0000060195F0000F18BF704703F000465200AF
:108D100043EB030313F4801F08BF013DF7D043EA80
:108D20000603704794EA0C0F0CEA135518BF95EA36
:108D30000C0F0CD050EA410618BF52EA4306D1D1BD
:108D400081EA030101F000414FF0000070BD50EADC
:108D5000410606BF1046194652EA430619D094EA66
:108D60000C0F02D150EA013613D195EA0C0F05D150
:108D700052EA03361CBF104619460AD181EA0301A4
:108D800001F0004141F0FE4141F470014FF000005C
:108D900070BD41F0FE4141F4780170BD70B54FF0F7
:108DA000FF0C4CF4E06C1CEA11541DBF1CEA135577
:108DB00094EA0C0F95EA0C0F00F0A7F8A4EB050459
:108DC00081EA030E52EA03354FEA013100F0888050
:108DD0004FEA03334FF0805545EA131343EA126319
:108DE0004FEA022245EA111545EA10654FEA0026CE
:108DF0000EF000419D4208BF964244F1FD0404F587
:108E0000407402D25B084FEA3202B61A65EB0305E2
:108E10005B084FEA32024FF480104FF4002CB6EB9F
:108E2000020E75EB030E22BFB61A754640EA0C001F
:108E30005B084FEA3202B6EB020E75EB030E22BF5F
:108E4000B61A754640EA5C005B084FEA3202B6EBA0
:108E5000020E75EB030E22BFB61A754640EA9C005F
:108E60005B084FEA3202B6EB020E75EB030E22BF2F
:108E7000B61A754640EADC0055EA060E18D04FEAED
:108E8000051545EA16754FEA06164FEAC30343EA8D
:108E900052734FEAC2025FEA1C1CC0D111F4801F5A
:108EA0000BD141EA00014FF000004FF0004CB6E753
:108EB00011F4801F04BF01430020B4F1FD0C88BFF2
:108EC000BCF5E06F3FF6AFAEB5EB030C04BFB6EBFD
:108ED000020C5FEA500C50F1000041EB045170BDF0
:108EE0000EF0004E4EEA113114EB5C04C2BFD4EB1D
:108EF0000C0541EA045170BD41F480114FF0000EA1
:108F0000013C90E645EA060E8DE60CEA135594EA1C
:108F10000C0F08BF95EA0C0F3FF43BAF94EA0C0F1F
:108F20000AD150EA01347FF434AF95EA0C0F7FF494
:108F300025AF104619462CE795EA0C0F06D152EAE8
:108F400003353FF4FDAE1046194622E750EA4106CC
:108F500018BF52EA43067FF4C5AE50EA41047FF4DD
:108F60000DAF52EA43057FF4EBAE12E74FF0FF3C42
:108F700006E000BF4FF0010C02E000BF4FF0010C13
:108F80004DF804CD4FEA410C7FEA6C5C4FEA430C8C
:108F900018BF7FEA6C5C1BD001B050EA410C0CBFDB
:108FA00052EA430C91EA030F02BF90EA020F00203D
:108FB000704710F1000F91EA030F58BF994208BFA4
:108FC00090422CBFD8176FEAE37040F00100704761
:108FD0004FEA410C7FEA6C5C02D150EA013C07D1B8
:108FE0004FEA430C7FEA6C5CD6D152EA033CD3D003
:108FF0005DF8040B704700BF8446104662468C46FD
:109000001946634600E000BF01B5FFF7B7FF00282F
:1090100048BF10F1000F01BD4DF808EDFFF7F4FF58
:109020000CBF012000205DF808FB00BF4DF808EDE3
:10903000FFF7EAFF34BF012000205DF808FB00BF06
:109040004DF808EDFFF7E0FF94BF012000205DF828
:1090500008FB00BF4DF808EDFFF7CEFF94BF0120DD
:1090600000205DF808FB00BF4DF808EDFFF7C4FFD6
:1090700034BF012000205DF808FB00BF4FEA410229
:10908000B2F1E04324BFB3F5001CDCF1FE5C0DD966
:1090900001F0004C4FEAC0024CEA5070B2F1004FB0
:1090A00040EB830008BF20F00100704711F0804FB3
:1090B00021D113F13872BCBF01F00040704741F478
:1090C00080114FEA5252C2F11802C2F1200C10FA7C
:1090D0000CF320FA02F018BF40F001004FEAC12360
:1090E0004FEAD32303FA0CFC40EA0C0023FA02F304
:1090F0004FEA4303CCE77FEA625307D150EA0133DA
:109100001EBF4FF0FE4040F44000704701F00040A9
:1091100040F0FE4040F40000704700BF80F0004087
:1091200002E000BF81F0004142001FBF5FEA41033F
:1091300092EA030F7FEA226C7FEA236C6AD04FEA3F
:109140001262D2EB1363C1BFD21841404840414084
:10915000B8BF5B42192B88BF704710F0004F40F436
:10916000000020F07F4018BF404211F0004F41F452
:10917000000121F07F4118BF494292EA030F3FD01E
:10918000A2F1010241FA03FC10EB0C00C3F1200331
:1091900001FA03F100F0004302D5494260EB4000C0
:1091A000B0F5000F13D3B0F1807F06D340084FEA2B
:1091B000310102F10102FE2A51D2B1F1004F40EB20
:1091C000C25008BF20F0010040EA03007047490088
:1091D00040EB000010F4000FA2F10102EDD1B0FA53
:1091E00080FCACF1080CB2EB0C0200FA0CF0AABF48
:1091F00000EBC25052421843BCBFD04018437047E6
:1092000092F0000F81F4000106BF80F400000132EB
:10921000013BB5E74FEA41037FEA226C18BF7FEAC2
:10922000236C21D092EA030F04D092F0000F08BF04
:109230000846704790EA010F1CBF0020704712F0EB
:109240007F4F04D1400028BF40F00040704712F12A
:1092500000723CBF00F50000704700F0004343F08F
:10926000FE4040F4000070477FEA226216BF0846C5
:109270007FEA23630146420206BF5FEA412390EA88
:10928000010F40F4800070474FF0000304E000BF7E
:1092900010F0004348BF40425FEA000C08BF70472F
:1092A00043F0964301464FF000001CE050EA0102F3
:1092B00008BF70474FF000030AE000BF50EA010208
:1092C00008BF704711F0004302D5404261EB4101F5
:1092D0005FEA010C02BF84460146002043F0B6431A
:1092E00008BFA3F18053A3F50003BCFA8CF2083A3F
:1092F000A3EBC25310DB01FA02FC634400FA02FC48
:10930000C2F12002BCF1004F20FA02F243EB02004E
:1093100008BF20F00100704702F1200201FA02FCB0
:10932000C2F1200250EA4C0021FA02F243EB0200A3
:1093300008BF20EADC7070474FF0FF0C1CEAD052E7
:109340001EBF1CEAD15392EA0C0F93EA0C0F6FD0A8
:109350001A4480EA010C400218BF5FEA41211ED086
:109360004FF0006343EA501043EA5111A0FB013172
:109370000CF00040B1F5000F3EBF490041EAD37147
:109380005B0040EA010062F17F02FD2A1DD8B3F1C3
:10939000004F40EBC25008BF20F00100704790F032
:1093A000000F0CF0004C08BF49024CEA502040EA84
:1093B00051207F3AC2BFD2F1FF0340EAC25070474A
:1093C00040F400004FF00003013A5DDC12F1190F88
:1093D000DCBF00F000407047C2F10002410021FAFA
:1093E00002F1C2F1200200FA02FC5FEA310040F112
:1093F000000053EA4C0308BF20EADC70704792F08B
:10940000000F00F0004C02BF400010F4000F013AC2
:10941000F9D040EA0C0093F0000F01F0004C02BFBD
:10942000490011F4000F013BF9D041EA0C018FE72C
:109430000CEAD15392EA0C0F18BF93EA0C0F0AD032
:1094400030F0004C18BF31F0004CD8D180EA010058
:1094500000F00040704790F0000F17BF90F0004FF1
:10946000084691F0000F91F0004F14D092EA0C0FD3
:1094700001D142020FD193EA0C0F03D14B0218BF66
:10948000084608D180EA010000F0004040F0FE40AC
:1094900040F40000704740F0FE4040F44000704748
:1094A0004FF0FF0C1CEAD0521EBF1CEAD15392EAC7
:1094B0000C0F93EA0C0F69D0A2EB030280EA010CB7
:1094C00049024FEA402037D04FF0805343EA111150
:1094D00043EA10130CF000408B4238BF5B0042F1AE
:1094E0007D024FF4000C8B4224BF5B1A40EA0C0053
:1094F000B3EB510F24BFA3EB510340EA5C00B3EB85
:10950000910F24BFA3EB910340EA9C00B3EBD10F72
:1095100024BFA3EBD10340EADC001B0118BF5FEAC4
:109520001C1CE0D1FD2A3FF650AF8B4240EBC250ED
:1095300008BF20F0010070470CF0004C4CEA5020AE
:109540007F32C2BFD2F1FF0340EAC250704740F4FD
:1095500000004FF00003013A37E792F0000F00F0EF
:10956000004C02BF400010F4000F013AF9D040EA6D
:109570000C0093F0000F01F0004C02BF490011F401
:10958000000F013BF9D041EA0C0195E70CEAD153F9
:1095900092EA0C0F08D142027FF47DAF93EA0C0FE0
:1095A0007FF470AF084676E793EA0C0F04D14B02C4
:1095B0003FF44CAF08466EE730F0004C18BF31F076
:1095C000004CCAD130F000427FF45CAF31F0004370
:1095D0007FF43CAF5FE700BF4FF0FF3C06E000BF09
:1095E0004FF0010C02E000BF4FF0010C4DF804CD2C
:1095F0004FEA40024FEA41037FEA226C18BF7FEA3C
:10960000236C11D001B052EA530C18BF90EA010F3D
:1096100058BFB2EB030088BFC81738BF6FEAE170CC
:1096200018BF40F0010070477FEA226C02D15FEA68
:10963000402C05D17FEA236CE4D15FEA412CE1D0D4
:109640005DF8040B704700BF844608466146FFE79B
:109650000FB5FFF7C9FF002848BF10F1000F0FBD7D
:109660004DF808EDFFF7F4FF0CBF012000205DF876
:1096700008FB00BF4DF808EDFFF7EAFF34BF0120FB
:1096800000205DF808FB00BF4DF808EDFFF7E0FF94
:1096900094BF012000205DF808FB00BF4DF808EDE5
:1096A000FFF7D2FF94BF012000205DF808FB00BF48
:1096B0004DF808EDFFF7C8FF34BF012000205DF82A
:1096C00008FB00BF4FEA4002B2F1FE4F0FD34FF04C
:1096D0009E03B3EB12620DD94FEA002343F000431F
:1096E00010F0004F23FA02F018BF404270474FF0CD
:1096F0000000704712F1610F01D1420205D110F054
:10970000004008BF6FF0004070474FF00000704706
:1097100042000ED2B2F1FE4F0BD34FF09E03B3EBDB
:10972000126209D44FEA002343F0004323FA02F007
:1097300070474FF00000704712F1610F01D14202F3
:1097400002D14FF0FF3070474FF00000704700BF6C
:1097500043F21003C2F200031868704720F00301BF
:1097600010F00300C0F1000051F8043B00F1040CBC
:109770004FEACC0C6FF000021CBF22FA0CF213432C
:109780004FF0010C4CEA0C2C4CEA0C4CA3EB0C02F5
:1097900022EA030212EACC1204BF51F8043B04305F
:1097A000F4D013F0FF0F1FBF013013F47F4F0130CF
:1097B00013F47F0F18BF0130704700BF4672657108
:1097C00075656E637920726573706F6E7365206660
:1097D0006F722044534F205175616400253264003C
:1097E0002532646B0000000025336400256400000E
:1097F0002064420044656700487A000023204672D6
:10980000657120202064422020202050686173650B
:1098100028646567290D0A002531306420253364EA
:109820002E253033642000002533642E2530326429
:109830000D0A000020202020202020202020202091
:109840002020202020202020202020202020202018
:109850002020202020202020202020202020202008
:1098600020202020202020202020202020202020F8
:109870002020202020202020202020004D65617302
:109880007572696E672E2E2E20686F6C64206B6572
:109890007920746F2061626F72742E2E2E2020202A
:1098A00000000000256420487A3A2056726D73202B
:1098B0002564206D56202064422025642E253032F8
:1098C00064202070686173652025642020202000BA
:1098D00041626F7274656421000000004D656E7511
:1098E0003A0000004661737400000000536C6F770B
:1098F0000000000044726177206F766572000000FE
:109900005361766520424D5000000000536176653A
:109910002043535600000000465245512530336421
:109920002E424D500000000057726974696E672026
:1099300025732E2E2E000000257320777269747413
:10994000656E2120202020004572726F7220777290
:109950006974696E672066696C652E2020000000BE
:1099600046524551253033642E43535600000000C3
:10997000424DF6BB00000000000076000000280009
:10998000000090010000F000000001000400000051
:10999000000080BB0000701700007017000010006E
:1099A00000000000000000002020202020202020B7
:1099B0002020202020202020202020204841524408
:1099C0004641554C542020202020202020202020BB
:1099D00020202020200000000A53503A20000000E0
:1099E000202050433A20000020204C523A20000012
:1099F0000A524547533A2072302000002C20723121
:109A0000200000000A2020202020207232200000A8
:109A10002C207233200000002C20723132200000F4
:109A20000A53434220484653523A20000A534342C5
:109A300020434653523A20000A535441434B20449A
:109A4000554D503A0A0000006C6F673130660000D7
:109A5000706F77660000000073717274660000001A
:109A60000000803F0000C03F00000000DCCFD13587
:109A70000000000000C0153F000FC93F000F494023
:109A800000CB9640000FC9400053FB4000CB16416D
:109A900000ED2F41000F49410031624100537B41ED
:109AA000003A8A4100CB9641005CA34100EDAF41F2
:109AB000007EBC41000FC94100A0D5410031E24108
:109AC00000C2EE410053FB4100F20342003A0A4259
:109AD0000083104200CB164200141D42005C23425A
:109AE00000A5294200ED2F4200363642007E3C425E
:109AF00000C74242000F4942A2000000F9000000E6
:109B0000830000006E0000004E00000044000000D2
:109B10001500000029000000FC00000027000000E4
:109B200057000000D1000000F500000034000000E4
:109B3000DD000000C0000000DB000000620000004B
:109B400095000000990000003C0000004300000068
:109B50009000000041000000FE00000051000000E5
:109B600063000000AB000000DE000000BB0000004E
:109B7000C500000061000000B700000024000000E4
:109B80006E0000003A000000420000004D0000009E
:109B9000D2000000E00000000600000049000000C4
:109BA0002E000000EA00000009000000D1000000C3
:109BB000920000001C000000FE0000001D000000DC
:109BC000EB0000001C000000B100000029000000B4
:109BD000A70000003E000000E80000008200000036
:109BE00035000000F50000002E000000BB00000062
:109BF0004400000084000000E90000009C00000018
:109C00007000000026000000B40000005F000000AB
:109C10007E000000410000003900000091000000BB
:109C2000D60000003900000083000000530000004F
:109C300039000000F40000009C00000084000000D7
:109C40005F0000008B000000BD000000F900000074
:109C5000280000003B0000001F000000F80000008A
:109C600097000000FF000000DE000000050000007B
:109C7000980000000F000000EF0000002F0000001F
:109C8000110000008B0000005A0000000A000000D4
:109C90006D0000001F0000006D0000003600000095
:109CA0007E000000CF00000027000000CB00000075
:109CB00009000000B70000004F000000460000004F
:109CC0003F000000660000009E0000005F000000F2
:109CD000EA0000002D0000007500000027000000D1
:109CE000BA000000C7000000EB000000E500000023
:109CF000F10000007B0000003D00000007000000B4
:109D000039000000F70000008A0000005200000047
:109D100092000000EA0000006B000000FB00000061
:109D20005F000000B10000001F0000008D00000077
:109D30005D00000008000000560000000300000065
:109D40003000000046000000FC0000007B00000026
:109D50006B000000AB000000F0000000CF0000002E
:109D6000BC000000200000009A000000F400000089
:109D7000360000001D000000A9000000E300000004
:109D800091000000610000005E000000E60000009D
:109D90001B000000080000006500000099000000A2
:109DA000850000005F00000014000000A00000001B
:109DB00068000000400000008D000000FF0000006F
:109DC000D8000000800000004D000000730000007B
:109DD000270000003100000006000000060000001F
:109DE0001500000056000000CA00000073000000CB
:109DF000A8000000C900000060000000E2000000B0
:109E00007B000000C00000008C0000006B00000020
:109E10000400000007000000090000000000C93F26
:109E20000000F0390000DA370000A2330000842E71
:109E30000000502B0000C2270000D0220000C41FE9
:109E40000000C61B00004417000000000000304363
:109E500000000000000030C33863ED3EDA0F493FD8
:109E60005E987B3FDA0FC93F6937AC3168212233F6
:109E7000B40F14336821A2331430002043000000D3
:109E800004000000DC0000001F00140001000000BE
:109E9000143000200000000000000000000000005E
:109EA00000000000000000000000000000000000B2
:109EB000000000007C9E020800000000000000007E
:109EC0000000000000000000000000000000000092
:109ED0000000000000000000000000000000000082
:109EE0000000000000000000000000000000000072
:109EF0000000000000000000000000000000000062
:109F00000000000000000000000000000000000051
:109F10000000000000000000000000000000000041
:109F20000000000000000000000000000000000031
:109F30000000000000000000000000000000000021
:109F40000000000000000000000000000000000011
:109F50000000000000000000000000000000000001
:109F600000000000000000000000000000000000F1
:109F700000000000000000000000000000000000E1
:049F800000000000DD
:0400000508025EADE2
:00000001FF
